:020000040000FA
:100000008A15CB205B213728F6000308F7000A0881
:10001000F8008A1183010317C830A000A00B0E2836
:10002000191B2D280313F00B2D287108F0007913EC
:100030007208F4007308F5006E08EF00EE0110106E
:100040000F08F2000E08F3000C1C2D28DD30F3071A
:100050000318F20A0B30F207EF0A031310148D1283
:1000600078088A0077088300F60E760E090029309A
:100070007E25F100F0001B307E25FB000A30EA00EF
:100080002830FD00E3014B2291225430A526AE30EA
:10009000D7265C30A926AC30D7264523C3258E0150
:1000A0008F018B13DD308E0703188F0A0B308F07FB
:1000B0000C10EE0A0319EE038B17E30A791B67286D
:1000C000EA0B6728B70A0319B60A2830EA00E70ADC
:1000D000E824D1244B229122D422D1242A23A32301
:1000E0005923E623F91CF522FD0B80208A15FD0813
:1000F00003192C218A11D124CF220C1C7D285128D0
:10010000FA1A0800F918080064189328E4180D2951
:1001100064191729E4197B29641ABD29E41AD7291F
:10012000641B222A08006A26DF20F8256C30A526E9
:100130003D274E30EB0004302B26F8251C307E2561
:10014000DD257030DD256830DD256F26FB1DC020E4
:10015000FB190021F825C8307426E71FB128EE20CE
:100160000800323098263D274A30EB0005302B2618
:10017000F8251C307E25DD251D307E25DD25080077
:10018000AC30A926AE30BE26ED263D277B18D528FB
:100190007910F91148308400FE25FE25FE25FE2544
:1001A000F325F8255730DD2508004A30EB000530EF
:1001B000641804302B26F8256B30DD25D228AE30AC
:1001C000A5263D2779104C308400FE25FE25F32519
:1001D000FB25F325F8255630DD250800203098262C
:1001E0002430B126E0263D274A307B184B30EB0007
:1001F00005302B26F8254130DD256830DD25080047
:10020000AC30A9263D274E307B184F30EB0005302F
:100210002B26F8254130DD2508006A26DF20F82549
:10022000C0206F260021C8307426EE2008006A2600
:100230008A3024268E3074261C307E25DD258025CC
:10024000DD256F26F825F825283098263D274B30E8
:100250007B184C30EB0006302B26CA3074269027D2
:100260003230A5260230C100E026BA1B74292008CE
:100270002404031D4629A11B4629A51B462921301C
:1002800098262530B126E02621304C2920309826AA
:100290002430B126E0262030BE2604272808031D7E
:1002A0005B29A91B5B292930BE26ED263330BE26EB
:1002B0003208BF0060292830BE26ED263230BE2627
:1002C000042799279930C100ED263D277910F911AF
:1002D00047307B1848308400FE25FE25F915FE25A1
:1002E000F325FB25F3250800F8252D30DD25DD2538
:1002F000DD25DD2508006A2699302426A230E71B7B
:10030000AB3024266F26203098262430B126E026F4
:1003100099270330C000E830C10004273A30B126E5
:10032000243098260427BA1BA62999272730C00015
:100330000F30C1007F263D277910F9114D30840020
:10034000FE25FE25F325FB25F325AD293930DD25D6
:10035000DD25DD25FB253930DD252530DD25CA30BD
:1003600074262430E71B203098263D274A307B181E
:100370004B30EB0006302B2608006A26B4302426CA
:100380006F262E30CD212C30CD213030A5263D27B3
:100390004E30EB0004302B260800A9263D274E30B6
:1003A0007B184F30EB0005302B26F82508006A2615
:1003B000F23024266F263830A5263D274E30EB003C
:1003C00004302B26F825323098263630BE260427F6
:1003D00099272430C100ED263D274C30EB00043036
:1003E0002B26F8258A3074263630A52699270E301C
:1003F000C0001030C10004273D2779104F30840021
:10040000FE25F325F8256830DD257230DD257330B3
:10041000DD25CA3074264230982699273C30C10029
:1004200004273D274F308400F325F3256D30DD256B
:10043000423098263D274F308400F325F325733052
:10044000DD2508006A26C53024268E3074261C302F
:100450007E25E03EDD258025DD256F26263097258B
:100460003D276F267910F9114D308400FE25FE25B9
:10047000FE25F325F82585244122F82579244122FB
:1004800008003D2779104A308400FE25FE25FE2510
:10049000FE25F3250800D801D901DA01DB01D401DA
:1004A000D5014030E6009D309F0075259F149F18B0
:1004B000572AA13075225A30BE26E3265A30D72655
:1004C0009F18602AA53075225830BE26E326583082
:1004D000D7269F18692A9D3075225430BE26E32600
:1004E0005430D726E60B572A08009F0094271E0891
:1004F000BC0083161E088312BD009F1408009F00D5
:100500002030E60090279F149F18842A83161E0D22
:100510008312C1001E0DC0009F14E326E60B842A3F
:10052000080099275830A5260330C000E326BB08F1
:10053000031DBD2A99270630C000E026BA1BBD2A3C
:100540004E30922552309725ED264430D92658302A
:10055000A52646309225E0264430BE26ED265C30A6
:10056000D9265C30A9269E2799270530C100E026B0
:10057000BA1FC72ADC01DD01C72A5A30A52644303C
:100580009225E0264E309225ED265C30D926543057
:10059000BE264A309725ED265430D9260800A530CE
:1005A0007F225430D726C7225430A5262A309225E0
:1005B000E026BA1FDC2ADF2AF91C08000028F918F7
:1005C0000800F91495018501870106170D30E9002F
:1005D00000307A2520309E250408E90BEB2AC3253C
:1005E000EC302426FF30EE0008005C30A9262C30C9
:1005F000C2267F263E3098262C30D7265C30A9268E
:100600002E30C2267F262E30D7266C30A5263830D5
:10061000BE267F263E3098263830D7267912F91A22
:10062000791690275630A5265430BE26E026F912BA
:10063000BA1BF916791A252BF91E252B5630A5263B
:100640003030BE267F263030D7265408D6005508D5
:10065000D70008005430A526A830B126E326A830DC
:10066000CA265C30A926A430B126E326A430CA26C7
:100670005B307E256305031D08004B23AC30D72675
:10068000A83098264B23AE30D7269427A830CA2608
:10069000A430CA2608005B307E25E800E80C031C65
:1006A00008000310BA1B0314BA0CBB0CBC0CBD0C25
:1006B0004E2B07306305031D0800AC30A92699278F
:1006C0008E30C0003630C100ED263A30C226BA1B4B
:1006D000722B20309826E3265C3089257F26203037
:1006E000CA267A2B24309826E0265C3089257F267E
:1006F0002430CA269027AC30A926AE30BE26ED267F
:10070000BA1B902B99270730C0000830C10004277E
:100710002830B126E3265C3089257F262830CA267A
:100720006C30A52699278E30C0003A30C100ED26E6
:100730003A30BE2632309826E3265C3089257F2663
:100740003230CA260800AF306E070318E22BAF30F4
:100750006F070318E22B791390278B137230A526AD
:100760007430BE266F088B17D300E0264B30CA26A4
:1007700090275308BD00F430C0002430C100ED269E
:100780004B30B126E32699270B30C100ED2699277F
:100790009730C10004273A30B126942754307E2583
:1007A000BA008025BB0004271C307E256B3C031D4E
:1007B000DC2B6C30D726080060309225ED266C309B
:1007C000D92608007917EC01ED010800A9307F2235
:1007D00066309225E026BA1B9427FA13BA1BFA1743
:1007E00064309225ED263B30BE263A08BF006330C8
:1007F00097257F26B030D72690272C309725FB1ED3
:10080000082CB030BE26ED264030D9264030A52633
:100810006C30BE26E026B830D72634309225ED263F
:100820003B30C226B630A526E3267224B630D72642
:10083000B830A92632309225ED269927C00A042720
:10084000B630BE26E326BA30CA2690272E3097252A
:100850007B1E312CB030BE26ED264030D9264030EC
:10086000A5265C30C226E026B830D726383092253F
:10087000ED263B30C226B230A526E3267224B230E4
:10088000D726BA30B1267F26BA30CA269027303014
:1008900092255430A526E026B830D7263A30922546
:1008A000ED263B30C226B430A526E3267224B430B0
:1008B000D726BA30B1267F26BA1B702C30307B0584
:1008C0000319642CFA1B702C403092257F263C08BB
:1008D00095009712BD1B971617123D1B171608009F
:1008E000950108003E3092257F263C3097257F26D3
:1008F00008009027323098262730C0001030C10001
:1009000004271E308925E3260800992720309826E1
:100910007B188F2C2730C0001030C100932C03307F
:10092000C000E830C100042722308925E3260800F2
:10093000EB000530E800473084006B08040203191F
:10094000A62C8008031DA62C840A9D2C461CAA2CCC
:100950002D30C5246B0A0402031DB02C2E30C52493
:1009600030300007C2000408C3007C08840042083D
:100970008000040AFC00430A8400513C0319C22C85
:10098000E80BAA2C0930C5240800C2000408C300E3
:100990007C08840042088000040AFC0043088400AC
:1009A00008007C0384000A30000203190800831643
:1009B000981CD82C8312840A00089900FC0A0A3C6F
:1009C000031908007C08840000089900FC0A08004C
:1009D000851D002DE5017A1E0800FA1AFB2CE7019F
:1009E0000310E40D031864145730791F59307E2525
:1009F00064050319ED2C013074267A12FA120800EE
:100A00007A16E50A03195C2DD8306507031D080026
:100A1000092DFA16641A4A2D852422307A253A3097
:100A20009E253C309E2579241E307A253A309E251D
:100A30003C309E259927203098261A307B180630A6
:100A4000BF00E026BA1B2D2D992726309725C10A15
:100A5000E32626307A253C309E251A30E9002030E6
:100A600084008001840AE90B312D5408B000550838
:100A7000B1000D30E90000307A2520309E250408B1
:100A8000E90B3E2DC32585307426D4302426FF3053
:100A9000EE000900AE01AF01AC01AD015408B00099
:100AA0005508B100B801B901C325DA302426D43085
:100AB0002426FF30EE00090026307A2520309E25BE
:100AC00022307A2520309E2520309E251E307A2522
:100AD00020309E2520309E25C325E6302426D430A4
:100AE0002426851D712DC32509001E30DE00DE0B76
:100AF000772D080003178D000313080003178D00DE
:100B0000031783168C130C1483120C088D0A03131D
:100B100008007E25BE008025BF008025C0008025FE
:100B2000C1000800BE01BF017A258D2D08007E2579
:100B3000BC008025BD00BA01BB01080084008B13F6
:100B400083168D128312F917031700088C00831681
:100B50008C130C1555308D00AA308D008C14630059
:100B600000008C18B12D0C11831203178D0A840A12
:100B700003130D12F91FBE2DF913A42D8D12831628
:100B80008D168312090003300711192656260330EB
:100B900019265E26033019265E26023019265E26A7
:100BA0002830DD252830DD250C30DD250130DD2520
:100BB00056260630DD2507150800E200F0308505D1
:100BC000620E0F3985040712E21B07166326F03008
:100BD000850562080F3985040712E2190716632696
:100BE0005E266208080030300007DD25840A080010
:100BF0002030DD2508002E30DD2508000008840A9D
:100C0000003E0319072E303EDD25791408007918BF
:100C1000162E00080319122E7914203046182D3094
:100C2000DD250800F9190C2EF82508003030DD25E7
:100C30000800E200F030850562080F3985040712CC
:100C4000E2190716632608007E25003E03190800F6
:100C5000DD258025252EE800473084006B0804023E
:100C600003193E2E0008031D3E2E0408523C680264
:100C70004618FF3E03193E2E840A2E2E7910461C7C
:100C8000452E2D30DD254610E8036B0804020319BC
:100C900079146B0A0402031D512EFB25E803031986
:100CA0000800FE25E80303190800452E2030DF0068
:100CB000E001E00B592EDF0B592E08006430E000F4
:100CC000E00B602E0800642E0714662E672E0710B6
:100CD000692E080007118030DD250715080007116F
:100CE000C030DD25071508000711DD2507150800B0
:100CF00056268519782E5626851D7B2E08003E081F
:100D0000C2003F08C3004008C4004108C500E026F7
:100D1000BA1F902E4230B126E3264230B126080099
:100D20004230B126E3263A30B126423098260800F8
:100D300084000008BA00840A0008BB00840A000886
:100D4000BC00840A0008BD0008008400BA01BB0191
:100D50009F2E8400BA01BB01801BBA03801BBB031A
:100D60009F2E84000008BE00840A0008BF00840A89
:100D70000008C000840A0008C10008008400BE0109
:100D8000BF01B82E8400BE01BF01801BBE03801BC3
:100D9000BF03B82E84003A088000840A3B08800014
:100DA000840A3C088000840A3D0880000800840012
:100DB000D12E84003A088000840A3B088000080095
:100DC000B427031808003A083E06D100782703101C
:100DD0003E083A06D11F803E0800D1019E27031C21
:100DE000B12703180800872794271F30D200C42793
:100DF000420D03187827031C3A0D03180800D20B84
:100E0000F72E5118A1270800D101410840043F04E2
:100E10003E04003C031C9E27031CB1270318080056
:100E2000C501C401C301C201C4271F30D200C427B9
:100E30003E084202031D262F3F084302031D262FB2
:100E400040084402031D262F41084502031C382F89
:100E50004108C5024008031C400FC4023F08031CA0
:100E60003F0FC3023E08031C3E0FC20203103D1495
:100E7000D20B172F5118A1270800D1019E27031864
:100E80000800CD272030D200BD0DBC0DBB0DBA0D22
:100E9000503084000A30D300800D0A30000203185D
:100EA00080008403D30B4C2FD20B442F51184614CF
:100EB00003100800D1002030D200463084005108D1
:100EC000D3000A300310840A03188007800CD30B68
:100ED000632FBA0CBB0CBC0CBD0CD20B5D2F0008F1
:100EE000FF3E031C3A0D031808004618A12708000E
:100EF0004108BD0740080318400FBC073F0803180E
:100F00003F0FBB073E0803183E0FBA0708003D0815
:100F1000C5003C08C4003B08C3003A08C2000800F2
:100F2000C101C001BF01BE01BD01BC01BB01BA01CD
:100F30000800C101C001BF01BE0108003A0D031C39
:100F400008003A088039BD09BC09BB09BA09BD0FC0
:100F5000AE2FBC0FAE2FBB0FAE2FBA0AD10A3A0785
:100F600008003E0D031C08003E088039C109C00975
:100F7000BF09BE09C10FC12FC00FC12FBF0FC12FA5
:100F8000BE0AD10A3E070800BD0DBC0DBB0DBA0D4F
:100F9000C50DC40DC30DC20D0800C601C701C801AF
:100FA000C901CA01CB01CC01CD01CE01CF01D001D5
:020FB000080037
:101000002010C529552A00282010E420613B6337B1
:10101000E4320000E529203AEE2AF4348039E5294B
:10102000203AE82BE5320036F029E53220326926F5
:10103000E936003A5328E123EE340000EE24533A17
:10104000E123EE340000ED2073384C10ED34F4341D
:101050000000EE24413AE123EE3400006F26A03B6D
:101060006F2B7436A0396926E936003AEE24563AD9
:10107000E123EE340000D424F232A036E126003C15
:10108000D424F232A036E9260037E126203C682A33
:101090006F39743A65360000E529203AD011EC37F3
:1010A000F3320000652D6F394110F0368039E529A3
:1010B000203A53297534743700006F2B743653105F
:1010C000EE32E5390000E529203A6129693A803796
:1010D000F620F232E730EE348033E529203A6129F8
:1010E00067378032E126EE344410F3346C38F9303F
:1010F0000000E5296939EC304F10F43A7538003AB0
:10110000E529203A6F2A443AF334003AE529203A97
:101110006F2A413A72348039E529203A6F2A433ADE
:10112000E33C0000F520203C6F2B7436E730803222
:10113000F520203C682A6539E8390000ED20733835
:101140004C10ED34F4340010F029E53220326926D9
:10115000E936003AE6272033201020102010001036
:10116000E12B743A8039ED20733800106924E8339C
:1011700028102E18C11880146F26A03B3014301789
:10118000C11880146D10E8278036A0187A2400005A
:10119000A01A7A240000850186018316F8308500A4
:1011A0008F308600CA3087004530810020309F0094
:1011B0008312031707309F00A0309E000313813075
:1011C0009F0003179530990084309800031383160D
:1011D0008D160D16FF30B200B400B6002630980010
:1011E0008130990083129817113090000C309700CD
:1011F000043092009501FF30EE000130E400F90167
:10120000FA01F91640308B0006130530E8008A1504
:101210000C1C08290C10E80B08298A11C3256A2622
:10122000683024266F26793024263C30E7008A1562
:101230000C1C18290C10E70B18298A111A30E90028
:101240002030840000307A258A1180258000840AAD
:101250008A15E90B2429080028307B190830FD0085
:101260008A11BE30FC00203098262430B126E026BA
:101270003D274A307B184B309824AE30A5263D27B9
:101280004E309824AC30A9263D274E307B184F3085
:1012900098246C30A5263D274E309824323098266D
:1012A0003D274A309824FC030D30C5240A30C5245C
:1012B000BE30FC0008004B30DF2603199621453074
:1012C000DF260319AC215330DF260319FA214F30F2
:1012D000DF260319D921851D222ABE308400413022
:1012E0008000840A68308000840A09308000840A03
:1012F00056308000840A09308000840A4130800022
:10130000840A09308000840A53308000840A09303E
:101310008000840A44308000840A0D308000840AF2
:101320000A308000BE30FC008A1108008A11C325F3
:101330005630DD25F82578264B225430BE269427DA
:101340000E30BA001030BB0004274A307A253C30FA
:101350009E258A15B82408008A11C3254F30DD2543
:101360005330DD2578268A15432746307A255830B4
:101370009E2544307A255A309E256F264430972585
:101380003D274C308400F325F325F325F325F32581
:10139000F325F825F825463097253D274C30840065
:1013A000F325F325F325F325F325F32578268A1570
:1013B00008008A11C3253130DD253030DD25F825C0
:1013C0004130DD2578268A1543275A30A52644303A
:1013D0009225E0269E273C30BE2694270330BA0093
:1013E000E830BB0004274E307A253C309E258A1514
:1013F000632408008A11C3255230DD256130DD25C4
:101400007430DD256930DD256F30DD2578268A15BD
:1014100043275830A52646309225E0265830D72657
:101420005A30A52644309225E0269927BF0AED269A
:101430005830C226042752307A253C309E258A1522
:10144000F724080000300F2778268A1547227822D3
:10145000A6222E238723972504300F278A15E826F6
:1014600003196D296E253A2561244F24B6242D24B5
:10147000CE2209236223AA23CF23D923E323F524F1
:10148000C025E9252F2659268A26ED236D290A3005
:101490000F276F261C307E25DD258025DD258A154A
:1014A000E826031908008A116F260D3074261C30B7
:1014B0007E25DD258025DD258A15E826031D08000B
:1014C0001C308A117E258A156B3C031D6C2A6D30F9
:1014D000C4006930C500702A6B30C4006D30C5008F
:1014E0008A111C307A2544309E258A15532A08001B
:1014F0000F300F276F26543097253D274D3084003D
:10150000F325F325F325F325F8256D30DD25DD25BD
:101510008A15E8260319080038270D3032274D3088
:10152000CD26C13032274E30CD26C23032274F3043
:10153000CD26C33032275030CD268A110A305A27A3
:1015400054307A253C309E258A15080014300F2728
:101550006F262C3097253D274D308400F325F32549
:10156000F8251C307E25DD257030DD256830DD2531
:101570008A15E8260319080038270D3032274D3028
:10158000CD26C13032274E30CD268A110A305A2757
:101590002C307A253C309E258A1508001A300F27FA
:1015A0003230922594277430BC006A30BD00ED269D
:1015B0003D276F2647308400F325FB25F325F325CF
:1015C000F8255630DD252F30DD251C307E25DD2524
:1015D0007030DD256830DD258A15E82603190800FE
:1015E000C23032270D3032274830CD26C330322763
:1015F0004930CD268A110A305A2799277430C00005
:101600006A30C100042732307A253C309E258A1585
:1016100008001E300F276F26343097253D274E30A7
:101620008400F325F325F3258A15E826031908001D
:1016300038270D3032274E30CD26C13032274F307B
:10164000CD26C23032275030CD268A110A305A2793
:1016500034307A253C309E258A15080023300F2728
:101660001B307E25FB006F262E3097253D274C3002
:101670008400F325F325F32530307B18DD25F8258C
:101680004130DD258A15E8260319080038270D307A
:1016900032274C30CD26C13032274D30CD26C230D6
:1016A00032274E30CD268A110A305A2799274E30DC
:1016B000C0002030C1007F262E307A253C309E2588
:1016C0008A15080029300F276F26383097253D27C7
:1016D0004E308400F325F325F3258A15E8260319F7
:1016E000080038270D3032274E30CD26C130322742
:1016F0004F30CD26C23032275030CD268A110A30E5
:101700005A2738307A253C309E258A1508002E301D
:101710000F276F26303097253D274D308400F32565
:10172000F325F8255630DD258A15E826031908002B
:1017300038270D3032274D30CD26C13032274E307C
:10174000CD268A110A305A2730307A253C309E2522
:101750008A15080036300F276F263A3097253D2727
:101760004E308400F325F325F3258A15E826031966
:10177000080038270D3032274E30CD26C1303227B1
:101780004F30CD26C23032275030CD268A110A3054
:101790005A273A307A253C309E258A1508003B307E
:1017A0000F278A153C30F723E826031908003C3040
:1017B0000C2C40300F278A153E30F723E8260319FA
:1017C00008003E300C2C45300F278A154030F72397
:1017D000E8260319080040300C2C98300F278A1592
:1017E0006630F723E8260319080066300C2C8A11AE
:1017F000972599271D30C000CD30C100ED263D272B
:101800006F2648308400F325FB25F325F325F825C2
:101810005630DD258A1508003F2738270D3032273E
:101820004830CD26C23032274930CD26C33032274A
:101830004A30CD268A110A305A2799271D30BE001A
:10184000CC30BF007F2699271D30C000CD30C100AD
:1018500004273C309E258A1508004C300F276F2640
:10186000902729307E25BD003D274F308400F32589
:10187000F3258A15E8260319080038270D3032278A
:101880004F30CD26C13032275030CD268A110A3054
:101890005A2728307A253C309E258A150800523078
:1018A0000F278A15E826031908008A1543274430B4
:1018B0007A255A309E2546307A2558309E258A153D
:1018C000080057300F278A111D30BA00CD30BB00F9
:1018D0006530BC000030BD004E30922504273D2706
:1018E0006F264C3084007B18FB25F3257B1CFB25E1
:1018F000F325F325F3258A15C23013278A15E82628
:1019000003190800C0307B18C13032270D30322750
:101910004C30CD26C23032274D30CD26C330322751
:101920004E30CD26C43032274F30CD268A110A30B2
:101930005A2799270130BF008630C0008C30C10083
:101940007F2699271D30C000CE30C1007F261D3074
:10195000BA00CD30BB006530BC000030BD000427AC
:101960004E307A253C309E258A1508005D300F27C1
:101970008A114A30972599270730C000D030C1001E
:10198000ED263D276F2649308400F325F325FB25FE
:10199000F325F325F8255630DD252F30DD2556308B
:1019A000DD258A15E8260319080038270D3032276F
:1019B0004930CD26C13032274A30CD26C3303227B8
:1019C0004B30CD26C43032274C30CD268A110A3018
:1019D0005A2799270730C000D030C10004274A3069
:1019E0007A253C309E258A15080063300F278A111E
:1019F00090273B30BC009B30BD0052309225ED2635
:101A00003D276F2647308400F325FB25F325F3257A
:101A1000F325F325F8254C30DD254730DD252F3023
:101A2000DD254830DD254730DD258A15E8260319F8
:101A30000800C23032270D3032274830CD26C3305F
:101A400032274930CD26C43032274A30CD26C53022
:101A500032274B30CD268A110A305A2799273B303E
:101A6000C0009B30C100042752307A253C309E25AF
:101A70008A15080068300F276F2690275B307E2577
:101A8000C1008A150310C10C031C482DBD0A422D4C
:101A90008A113D2750308400F3258A15E826031962
:101AA0000800C03032270D3032275030CD268A1141
:101AB0000A305A27BD080319BD0A99270730C1000B
:101AC0007F2699278A150314C10DBD0B632D8A113A
:101AD0005A307A2540309E258A1508006D300F2730
:101AE0006F261B307E25FB008A157B1C94257B18F6
:101AF00091258A15E8260319080038270D3032276A
:101B00007B1C94257B1891258A15E826031D080067
:101B10000130FB068A111A307A257A309E258A1503
:101B20007D2DB63013270800BC3013270800723013
:101B30000F276F261B307E25FB008A15FB1DBA255B
:101B4000FB19BD258A15E8260319080038270D3032
:101B50003227FB1DBA25FB19BD258A15E826031D72
:101B600008000830FB068A111A307A257A309E2543
:101B70008A15A62DB03013270800B33013270800AC
:101B800079300F276F261B307E25FB008A157B1DC1
:101B9000E6257B19E3258A15E8260319080038276E
:101BA0000D3032277B1DE6257B19E3258A15E826B3
:101BB000031D08000430FB068A111A307A257A309A
:101BC0009E258A15CF2DC83013270800C53013274E
:101BD000080080300F273230982699272730C00020
:101BE0001030C10004274230CA261E308925E32662
:101BF0006F263D274A308400F325F325F325F3258E
:101C0000F325F8251C307E25DD251D307E25DD25BC
:101C10001E307A258A15E8260319080038270D306A
:101C200032274A30CD26C13032274B30CD26C23044
:101C300032274C30CD26C33032274D30CD26C4302C
:101C400032274E30CD268A110A305A274230B1262B
:101C5000E0263A309E253C309E258A1508008630C5
:101C60000F272030982699278A157B183C2E27307D
:101C7000C0001030C100402E0330C000E830C10069
:101C80008A1104274230CA2622308925E3266F268E
:101C90003D274A308400F325F325F325F325F3256A
:101CA000F8254130DD256830DD2522307A258A157A
:101CB0000A2E8C300F276F26263097253D274D3072
:101CC0008400F325F325F325F325F8254330DD259E
:101CD0007930DD256330DD258A15E82603190800F3
:101CE00038270D3032274D30CD26C13032274E30C7
:101CF000CD26C23032274F30CD26C3303227503068
:101D0000CD268A110A305A2726307A253C309E2566
:101D10008A15080092300F276F261B307E25FB00A6
:101D20008A157B1AC126FB1AC5267B1A9A2EFB1A26
:101D30009A2EC9268A15E8260319080038270D307F
:101D400032277B1AC126FB1AC5267B1AAA2EFB1A3C
:101D5000AA2EC926E826031D080030307B0503198A
:101D6000B62E7B1AB82EFB127B12BA2E7B16BA2E19
:101D7000FB167B128A111A307A257A309E258A1535
:101D80009E2E9E3013278A150800A43013278A152B
:101D90000800AA3013278A1508008400E826031DCE
:101DA0000800800A0A300002031CD72E8001303060
:101DB00000078A11DD25103074268A15CE2EC50045
:101DC0008A117E25E80045037E2568048A150800EF
:101DD000E5018A1156268A158519E82E8A1156269C
:101DE0008A1585190A2FE50FEE2E8A11CE3074263A
:101DF0004F30DD254B30DD258A158A1156268A1590
:101E0000851DFD2E03118A11CE307426F825F82584
:101E10008A1508008A1156268A1503150800E8005D
:101E20008A11C325680803178D0008308F008A11B6
:101E300083168C170C140000000083120C0D0E0D7D
:101E400003137F3903190800DD2503170C0803135A
:101E50007F3903190800DD2503178D0A03188F0A3F
:101E60008A15172F07118A11DD258A150715080015
:101E700007118A11C030DD2507158A1508000317E0
:101E80008D00031308008A119027A430CA26A830B9
:101E9000CA264030E3008A114B225830BE26A430B7
:101EA0009826E326A430CA265A30BE26A8309826A3
:101EB000E326A830CA268A15E30B4B2F8A11A430DB
:101EC000982699274030C100042799272030C10067
:101ED000E0265830D726A830982699274030C100F0
:081EE00004275A30D726080040
:02400E009237E7
:1042000000000000000000000000000000000000AE
:10421000000000000000000000000000000000009E
:104220007F00FF0000000000000000000000000010
:1042300000000000000006006B006D0000000000A0
:10424000000000000000000000000000000000006E
:10425000000001000500DC002600AC00130088000F
:1042600007006C000B0018000000C8000300E80005
:1042700001002C0003002000C2008F0019009900EB
:10428000FF0000004F00530000000000000000008D
:104290006B005600000000006B00410000000000B1
:1042A0006B00520019009A0008001B0000007F00FC
:1042B00000003F0000001F00770035009300FF0062
:1042C0009F001200FF00FF000100AE00330033002A
:1042D00054006800650020004300790063006C0012
:1042E000650041006E0061006C007900730074008D
:1042F00000002000200020005600650072007300BE
:1043000069006F006E00200032002E003100200096
:104310002000000057006100740074002D00680048
:1043200072007300200020002000570068002F005A
:104330000000250052006500670065006E00200047
:104340002000000052006500670065006E0020003C
:104350004100680000002000200046007700640053
:10436000200041006800000041006D0069006E00FF
:104370002000200041006D00610078002000200036
:1043800056006D0069006E00000043007900630074
:104390006C00200054006F00740041006800200091
:1043A00054006F0074000000520065007300650047
:1043B000740000005000650061006B002000530095
:1043C0007400610074007300200000004600750056
:1043D0006C006C00200000004C006F007700200093
:1043E000560000004D00610078005300200041009D
:0A43F0007600670053002000000073
:00000001FF
